:020000040000FA
:10000000F728FA308C00811F0328811B05288C0BF0
:100010000328003405308C000328081508190E2821
:1000200009080800C13088000D2092000034C93052
:1000300088000D209C00003482078834DB34A23411
:100040009234D13494348434DA3480349034AC34FF
:10005000E034960003109C309607970A03182A286C
:100060006430960797030310F6309607980A031832
:10007000332816080A3E9900980300340A30950088
:10008000970198019901122012089A0003101C3060
:100090009A0703185A28323003109A070318642865
:1000A000323003109A0703186E2812089B000130A3
:1000B0009D00B428033097079A0112089A0069300E
:1000C0009A071A089B005728023097079A011208CE
:1000D0009A009B309A071A089B005728013097070F
:1000E0009A0112089A00CD309A071A089B005728E7
:1000F00005309D000B30950097019801990117205C
:100100001C089A0003101C309A07031894283230F8
:1001100003109A0703189E28323003109A07031819
:10012000A8281C089B00B428033097079A011C08D4
:100130009A0069309A071A089B00B4280230970782
:100140009A011C089A009B309A071A089B00B42851
:10015000013097079A011C089A00CD309A071A08B7
:100160009B00B4280516C0283230900017201C08C8
:100170009E001220031012091C070318B228051252
:100180001B081B0732308E08292017081C20051178
:10019000851586000A20FF30860018081C200515EA
:1001A000851186000A20FF30860019081C200511E1
:1001B000851186000A20FF30860015081C200515D1
:1001C000851586000A20FF3086008E0BC428172074
:1001D0001E0903101C07031878281C0903101E07AA
:1001E00003187828900BB6289D0B7A283E28831692
:1001F000C030810002308800003086000330850066
:1002000083128C0181013E28FF3FFF3FFF3FFF3FEC
:10021000FF3FFF3FFF3FFF3FFF3FFF3FFF3FFF3FEE
:10022000FF3FFF3FFF3FFF3FFF3FFF3FFF3FFF3FDE
:10023000FF3FFF3FFF3FFF3FFF3FFF3FFF3FFF3FCE
:10024000FF3FFF3FFF3FFF3FFF3FFF3FFF3FFF3FBE
:02400E00F93F78
:08400000FF3FFF3FFF3FFF3FC0
:00000001FF
